:020000040000FA
:0400000006EF00F017
:0800080030EF00F08A6AF00EEF
:10001000936E0F0EC16E956A8C6A966A8D6A84849F
:10002000386A396A3B6A3A6AD08EF28EF28CF2866E
:10003000F19EF1800E0E3B6E816E83EC00F00D0E92
:100040003B6E816E83EC00F00B0E3B6E816E83EC99
:1000500000F0070E3B6E816E83EC00F01AEF00F0AB
:10006000F2A0100081500000F00B396E393A3A626C
:100070004AEC00F0386E8DEC00F0836E76EC00F008
:1000800076EC00F076EC00F076EC00F076EC00F028
:10009000F29010003BB055EF00F039A0010C39A2EE
:1000A000020C39A4030C39A60A0C3BB260EF00F035
:1000B00039A0040C39A2050C39A4060C39A60B0C86
:1000C0003BB46BEF00F039A0070C39A2080C39A43F
:1000D000090C39A60C0C3BB6000C39A0000C39A257
:1000E000000C39A4000C39A60D0C000CFA0E256E7C
:1000F000FA0E266E00000000262E7AEF00F0252E64
:1001000078EF00F01200FA0E246E000000000000EC
:100110000000242E85EF00F01200010EFA6E385018
:1001200038242A0FD8B0FA2AF96E3F0C060C5B0C63
:100130004F0C660C6D0C7D0C070C7F0C6F0C770C54
:0A0140007C0C390C5E0C790C710C7C
:020000040030CA
:04000000000C1F1EB3
:02000500038175
:060008000FC00FE00F40E5
:00000001FF
